:100000000C9434000C9451000C9451000C94510049
:100010000C9451000C9451000C9451000C940E015E
:100020000C9451000C9451000C9451000C94DD0080
:100030000C9451000C9451000C94AC000C945100A1
:100040000C9451000C9451000C9451000C945100EC
:100050000C9451000C9451000C9451000C945100DC
:100060000C9451000C94510011241FBECFEFD8E026
:10007000DEBFCDBF11E0A0E0B1E0E6E1F6E002C0F6
:1000800005900D92A031B107D9F711E0A0E1B1E0E0
:1000900001C01D92A531B107E1F70E945C010C94EB
:1000A00009030C9400000F931F93CF93DF93EC018F
:1000B00001E010E020E030E040EA50E4688179811E
:1000C0008A819B810E94F00187FD02C000E010E060
:1000D0001D830C838E859F858230910561F083306E
:1000E000910599F00197C9F416BC80916E00826069
:1000F00080936E0016C0109285001092840080914B
:100100006F00826080936F000CC01092B2008091EB
:10011000700082608093700004C081E090E00E94D3
:10012000090378949FB7F894809112019FBF8823A8
:10013000C9F310921201EA85FB858C819D81892B80
:1001400019F08081826002C080818D7F8083DF9181
:10015000CF911F910F9108951F920F920FB60F929A
:1001600011242F933F938F939F938091100190912F
:100170001101019690931101809310018091120159
:10018000813091F020911001309111018091130183
:10019000909114012817390738F081E080931201FB
:1001A00010921101109210019F918F913F912F9108
:1001B0000F900FBE0F901F9018951F920F920FB6C1
:1001C0000F9211242F933F938F939F93809110014F
:1001D00090911101019690931101809310018091EB
:1001E0001201813091F02091100130911101809124
:1001F0001301909114012817390738F081E080939A
:10020000120110921101109210019F918F913F9154
:100210002F910F900FBE0F901F9018951F920F9265
:100220000FB60F9211242F933F938F939F9380913A
:10023000100190911101019690931101809310018A
:1002400080911201813091F02091100130911101C3
:1002500080911301909114012817390738F081E03B
:100260008093120110921101109210019F918F91B1
:100270003F912F910F900FBE0F901F901895FC018A
:10028000219A85E290E09387828785B5836085BD5A
:1002900081E090E09587848722E030E0309314017C
:1002A0002093130124B5226024BD29EF27BD978731
:1002B000868780E090E00895CF92DF92EF92FF92E0
:1002C00080E091E00E943F01C12CD12C760160E0DA
:1002D00070E0CB01609300017093010180930201F3
:1002E0009093030180E091E00E9453008FEFC81AC1
:1002F000D80AE80AF80AC701B6010E94F4012FE6FD
:1003000032E143E05BE30E94A60220E030E0A90175
:100310000E948C01DFCF5058BB27AA270ED0DCC02B
:10032000CDD030F0D2D020F031F49F3F11F41EF444
:10033000C2C00EF4E095E7FBB8C0E92FDED080F331
:10034000BA17620773078407950718F071F49EF5D2
:10035000F6C00EF4E0950B2EBA2FA02D0B01B901BB
:1003600090010C01CA01A0011124FF27591B99F02B
:10037000593F50F4503E68F11A16F040A22F232F37
:10038000342F4427585FF3CF469537952795A79587
:10039000F0405395C9F77EF41F16BA0B620B730B2E
:1003A000840BBAF09150A1F0FF0FBB1F661F771F9F
:1003B000881FC2F70EC0BA0F621F731F841F48F454
:1003C000879577956795B795F7959E3F08F0B3CFDA
:1003D0009395880F08F09927EE0F979587950895C4
:1003E00040D008F481E00895E89409C097FB3EF4FA
:1003F00090958095709561957F4F8F4F9F4F992372
:10040000A9F0F92F96E9BB279395F69587957795EF
:100410006795B795F111F8CFFAF4BB0F11F460FFAF
:100420001BC06F5F7F4F8F4F9F4F16C0882311F007
:1004300096E911C0772321F09EE8872F762F05C01B
:10044000662371F096E8862F70E060E02AF09A95B6
:10045000660F771F881FDAF7880F9695879597F9AB
:100460000895990F0008550FAA0BE0E8FEEF161645
:100470001706E807F907C0F012161306E407F50798
:1004800098F0621B730B840B950B39F40A2661F00C
:10049000232B242B252B21F408950A2609F4A140AF
:1004A000A6958FEF811D811D089597F99F6780E8BC
:1004B00070E060E008959FEF80EC089500240A94B6
:1004C0001616170618060906089500240A9412162F
:1004D0001306140605060895092E0394000C11F462
:1004E000882352F0BB0F40F4BF2B11F460FF04C00F
:1004F0006F5F7F4F8F4F9F4F089557FD9058440F68
:10050000551F59F05F3F71F04795880F97FB991F72
:1005100061F09F3F79F0879508951216130614062F
:10052000551FF2CF4695F1DF08C0161617061806BC
:10053000991FF1CF86957105610508940895E89497
:10054000BB2766277727CB0197F908950BD0C4CF37
:10055000B5DF28F0BADF18F0952309F0A6CFABCFAE
:100560001124EECFCADFA0F3959FD1F3950F50E091
:10057000551F629FF001729FBB27F00DB11D639F55
:10058000AA27F00DB11DAA1F649F6627B00DA11DFB
:10059000661F829F2227B00DA11D621F739FB00DA1
:1005A000A11D621F839FA00D611D221F749F332711
:1005B000A00D611D231F849F600D211D822F762FAA
:1005C0006A2F11249F5750408AF0E1F088234AF0A7
:1005D000EE0FFF1FBB1F661F771F881F91505040F3
:1005E000A9F79E3F510570F060CFAACF5F3FECF3B3
:1005F000983EDCF3869577956795B795F795E795DF
:100600009F5FC1F7FE2B880F911D9695879597F9EF
:060610000895F894FFCFED
:100616000000000001006F12033B00000000000014
:00000001FF
